:100000001FC016C115C114C113C112C111C110C145
:10001000A0C00EC10DC10CC10BC10AC109C108C1EC
:1000200007C106C105C104C103C102C101C100C1AC
:10003000FFC0FEC03F003F2900023A3F293F2B800E
:1000400011241FBECFEFCDBFDFE3DEBFE4E3F0E05E
:1000500040E017C0B591A59135912591059107FD17
:100060000CC095918591EF01F92FE82F05900D9225
:10007000A217B307D9F7FE0104C01D92A217B30758
:10008000E1F7E034F40731F703D0A2C0F894FFCFD2
:1000900077D0E0E0F4E080818260808380818F7798
:1000A000808380818F7D808380818F7E808397D0C5
:1000B000A2D037D0ACD082D0B6D0D82F96D0A1D095
:1000C00030D0ABD07BD0AFD0C82F85E19FE308D034
:1000D0008D2F6AD080E09FE303D08C2F65D0E7CFCF
:1000E000EF92FF920F931F93CF93DF938C017C01CC
:1000F000C0E0D0E005C0F70181917F0155D0219685
:10010000F80101900020E9F73197E01BF10BCE17C1
:10011000DF0788F3DF91CF911F910F91FF90EF9050
:02012000089540
:100122001092293F10922A3F7894E0E0FAE081E0B1
:100132008287118281858E7F818788E290E086A303
:1001420097A3808186608083808181608083089507
:100152008F938FB78F939F93F8948091293F9091BB
:100162002A3F01968093293F90932A3F81E0809312
:0E0172000B0A78949F918F918FBF8F911895F3
:10018000E0E2F4E08081877F8083808184608083E7
:10019000E0E0F8E08DE695E08087918783E0878353
:0801A0008681806486830895C6
:1001A800E0E0F8E0948195FFFDCFE0E0F8E082839D
:0401B80083830895A0
:1001BC00F894E0E0FAE080818E7F808385818C600A
:0401CC00858308958A
:0E01D000EC0130D02ED0CE012ED0CE012DD09D
:0C01DE00E0E0F4E0808585FDFDCF089591
:0C01EA00E0E0F4E0808584FDFDCF089586
:0C01F600E0E0F4E08481826084830895DE
:0C020200E0E0F4E084818D7F84830895A7
:0C020E00E0E0F4E080858823ECF7089520
:0C021A00E0E0F4E080858823ECF3089518
:0A0226008091293F90912A3F08952E
:02023000E7CE17
:0202320008952D
:0202340008952B
:02023600089529
:0202380029DFBC
:10023A000D0A427265616B2054696D652831304B35
:05024A00687A293A006A
:10024F000D0A4D616B652054696D652831304B681F
:04025F007A293A00BE
:00000001FF
